:020000040800F2
:1000000000200020F90A0008E5070008E7070008BB
:1000100000000000000000000000000000000000E0
:10002000000000000000000000000000E9070008D8
:100030000000000000000000EB070008ED070008CA
:10004000490B000800000000490B0008490B00089C
:10005000490B0008490B0008F907000803080008CD
:10006000000000000D0800081D080008490B0008EA
:10007000490B0008490B0008490B0008000000006C
:10008000490B00080000000000000000490B0008B8
:1000900000000000490B0008490B0008490B00084C
:1000A000490B0008490B0008490B000835080008F7
:0800B000490B000800000000EC
:1000B80010B5064C2378002B07D1054B002B02D036
:1000C800044800E000BF0123237010BD5000002049
:1000D80000000000D0410008044B10B5002B03D0ED
:1000E8000349044800E000BF10BDC04600000000FE
:1000F80054000020D04100080023C25C0133002ACC
:10010800FBD1581E7047000002B4714649084900E7
:10011800095C49008E4402BC7047C046002243086F
:100128008B4274D303098B425FD3030A8B4244D3B7
:10013800030B8B4228D3030C8B420DD3FF220902F9
:1001480012BA030C8B4202D31212090265D0030BB8
:100158008B4219D300E0090AC30B8B4201D3CB03AE
:10016800C01A5241830B8B4201D38B03C01A5241F0
:10017800430B8B4201D34B03C01A5241030B8B42F2
:1001880001D30B03C01A5241C30A8B4201D3CB02DD
:10019800C01A5241830A8B4201D38B02C01A5241C2
:1001A800430A8B4201D34B02C01A5241030A8B42C5
:1001B80001D30B02C01A5241CDD2C3098B4201D3DD
:1001C800CB01C01A524183098B4201D38B01C01A5B
:1001D800524143098B4201D34B01C01A52410309D2
:1001E8008B4201D30B01C01A5241C3088B4201D381
:1001F800CB00C01A524183088B4201D38B00C01A2E
:10020800524143088B4201D34B00C01A5241411A54
:1002180000D20146524110467047FFE701B5002061
:1002280000F0F0F802BDC0460029F7D076E7704725
:1002380003460B437FD4002243088B4274D303093F
:100248008B425FD3030A8B4244D3030B8B4228D3E0
:10025800030C8B420DD3FF22090212BA030C8B4206
:1002680002D31212090265D0030B8B4219D300E0A6
:10027800090AC30B8B4201D3CB03C01A5241830B2B
:100288008B4201D38B03C01A5241430B8B4201D3DB
:100298004B03C01A5241030B8B4201D30B03C01A04
:1002A8005241C30A8B4201D3CB02C01A5241830A7E
:1002B8008B4201D38B02C01A5241430A8B4201D3AD
:1002C8004B02C01A5241030A8B4201D30B02C01AD7
:1002D8005241CDD2C3098B4201D3CB01C01A52413E
:1002E80083098B4201D38B01C01A524143098B42C7
:1002F80001D34B01C01A524103098B4201D30B01B0
:10030800C01A5241C3088B4201D3CB00C01A5241D4
:1003180083088B4201D38B00C01A524143088B4299
:1003280001D34B00C01A5241411A00D20146524132
:10033800104670475DE0CA0F00D04942031000D351
:100348004042534000229C4603098B422DD3030AA6
:100358008B4212D3FC22890112BA030A8B420CD3B6
:10036800890192118B4208D3890192118B4204D3DF
:1003780089013AD0921100E08909C3098B4201D35F
:10038800CB01C01A524183098B4201D38B01C01A99
:10039800524143098B4201D34B01C01A5241030910
:1003A8008B4201D30B01C01A5241C3088B4201D3BF
:1003B800CB00C01A524183088B4201D38B00C01A6C
:1003C8005241D9D243088B4201D34B00C01A524143
:1003D800411A00D20146634652415B10104601D3D0
:1003E8004042002B00D54942704763465B1000D35A
:1003F800404201B5002000F005F802BD0029F8D000
:1004080016E770477047C0461FB50C22002101A8A7
:1004180003F0D1FE8022184C184B120622610422E8
:10042800236080236261033A1B03A276E261220003
:10043800636000232C3213700722626322002000BD
:100448003C322383A360E3606362A3622363137077
:10045800E36400F0C9FB002801D000F0A5F9084BBF
:1004680020000193012301A9029300F027FD002831
:1004780001D000F099F91FBD6C0000200024014054
:100488000200000470B505008EB01422002103A8F4
:1004980003F091FE1822002108A803F08CFE264BD9
:1004A8002A689A4245D18023DB010893802308A853
:1004B8001B060C9301F0CAFE002801D000F074F965
:1004C80080201E4B4003196C00260143196401214A
:1004D8001A6C02400192019A5A6BA0200A435A638F
:1004E8005B6BC0050B400293029B022303935B18CE
:1004F80003A90493059601F049FA114C114B200009
:100508002360052363607B33236180336361802329
:10051800DB00A3612023E36180235B01A660E66022
:10052800236200F0D7FFB04201D000F03DF92C65FE
:10053800A5620EB070BDC046002401400010024004
:10054800D00000200800024007B501200C4A916B3A
:1005580001439163936B002203401100019308301B
:10056800019B00F02DFF092000F054FF00220A2013
:10057800110000F025FF0A2000F04CFF07BDC0461F
:1005880000100240F0B5022789B01422002103A808
:1005980003F011FE04210125A026474BF6055A6BEE
:1005A80030003A435A635A6B00243A400092009A4A
:1005B8005A6B0A435A635A6B0A400192019A5A6B62
:1005C8003E492A435A635B6B2A002B400293029BE5
:1005D80001F090FA30000022202101F08BFA2A0065
:1005E8002900374801F086FA364B03AA0393032300
:1005F800110033480493059401F0C8F9C0231B0285
:100608000393032303AA11002F480493059401F0D0
:10061800BDF92E4B300003930323049303AB190059
:10062800059401F0B3F904213000039103A904955E
:100638000594069401F0AAF908230393C423300013
:100648009B0303A90493059401F0A0F9C12330008A
:100658005B0103A9039304950594069701F096F9A5
:100668004023300003A903930494059401F08EF904
:1006780080230393882330005B0303A90493059424
:1006880001F084F903A90E4803950495059406948E
:1006980001F07CF922003900062000F091FE0620C6
:1006A80000F0B8FE22003900072000F089FE07207C
:1006B80000F0B0FE09B0F0BD0010024004180000C0
:1006C800000400503E0300000008005001810000B3
:1006D8000848094B10B5036003234360074BC36008
:1006E800074B836001F02AFA002801D000F05CF87B
:1006F80010BDC0462C01002000300040FF0F000054
:10070800B80B000010B592B03422002105A803F000
:1007180052FD1022002101A803F04DFD8020800029
:1007280001F046FA0A230593F63308930023099348
:100738000E9308330F9380239B024022109380234B
:1007480002240A929B053F3A05A80B920C940D943B
:10075800119301F059FA002801D072B6FEE7072379
:1007680003900490210001A80193029401F0ACFCCD
:10077800002801D072B6FEE712B010BD10B500F027
:1007880009FAFFF7BFFF03F01BFCFFF7FBFEFFF7BB
:10079800DBFEFFF739FE00F0B9F800F0F1F8FFF7DB
:1007A80097FF03F0EFFAFEE772B6FEE701200A4B67
:1007B80082B0196C0143196480211A6C4905024002
:1007C8000092009ADA6B0A43DA63DB6B0B40019301
:1007D800019B02B07047C04600100240FEE7FEE7EA
:1007E8007047704710B500F0E9F903F01BFC10BD25
:1007F80010B5082001F08EF910BD10B5802001F069
:1008080089F910BD10B5024800F086FF10BDC0463A
:10081800D000002010B5034800F07EFF024800F029
:100828007BFF10BD88010020E401002070B5134C47
:10083800200002F047FA10222368D96911421BD020
:100848000F4D1A622B78002B16D1200002F07CF98C
:100858000C4B0D481B685A6880235B429B1ADBB21D
:100868002B702A78094DD2B2290003F09BFC802214
:100878002900200002F064FE70BDC046400200203E
:100888007E06002088010020FE050020EA040020E2
:1008980070470000084B026882B09A4209D1802054
:1008A800064A0002116C01431164136C0340019362
:1008B800019B02B07047C046002000400010024073
:1008C80010B5040086B01422002101A803F073FCBF
:1008D8000C4B22689A4213D101200B4A516B0143F9
:1008E8005163536B01A903400093009B1023A02080
:1008F80001930E3B0293C0050233059301F046F8BD
:1009080006B010BD002000400010024010B588B0AD
:100918001C22002101A803F04EFC164C164B174A66
:1009280023600223636000232000A360E260236148
:10093800A36101F0BBFE002801D0FFF735FF2000BE
:1009480001F0DEFE002801D0FFF72EFF0022602311
:10095800200001A9019302920392059201F036FF4B
:10096800002801D0FFF720FF2000FFF7A9FF08B0FB
:1009780010BDC0463C01002000200040E7030000F5
:1009880010B5184B184C0C222360E1235B026360FE
:1009980000232000A360E36023616261A361E36137
:1009A80023626362A36202F041FD002801D0FFF7D1
:1009B800FBFE0021200002F03BFE002801D0FFF7DB
:1009C800F3FE0021200002F057FE002801D0FFF7B7
:1009D800EBFE200002F00EFE002801D0FFF7E4FE37
:1009E80010BDC046003801404002002070B5060026
:1009F8008EB01422002103A803F0DDFB1822002189
:100A080008A803F0D8FB334B32689A4260D101231F
:100A180008A8089301F01AFC002801D0FFF7C4FECB
:100A280080202D4BC001196C0025014319641A6CF4
:100A380002400192019A0222596B284811435963D6
:100A48005B6B03A913400293029BC0230492039398
:100A580005950695079500F099FF214C214B20003C
:100A68002360322363604E33236180235B01A560DA
:100A7800E5606561A561E561236200F02BFDA84290
:100A880001D0FFF791FE331DDC67A662164B174CA9
:100A98008022236033236360233BA3600023E36049
:100AA8006361A361E361802320005B01226123620B
:100AB80000F010FD002801D0FFF776FE1B20002271
:100AC8000121F467A66200F07BFC1B2000F0A2FC69
:100AD8000EB070BD00380140001002400004005004
:100AE800880100201C00024030000240E401002080
:100AF8000D488546FFF7CCFE0C480D490D4A0023EA
:100B080002E0D458C4500433C4188C42F9D30A4ABA
:100B18000A4C002301E013600432A242FBD303F025
:100B28001DFBFFF72BFEFEE7002000200000002041
:100B380050000020A042000850000020EC060020D1
:100B4800FEE7000070B5104B05001978002901D1A7
:100B5800012070BDFA208000FFF7E0FA0B4B01007E
:100B68001868FFF7DBFA00F061FC041EF0D1032DD2
:100B7800EED8020001202900404200F021FC044B7D
:100B880020001D60E5E7C0460400002000000020AA
:100B9800080000208023084A5B00116810B50B4349
:100BA80003201360FFF7CEFF041E03D1FFF7FEFDFD
:100BB800200010BD0124FBE700200240034A044B3B
:100BC80011681B785B1813607047C046D402002078
:100BD80004000020014B18687047C046D40200206A
:100BE80080684007C00F70470023F0B585B0040047
:100BF80001250393984200D1B7E0856D9D4205D148
:100C0800FFF740FC23005433E5651D7080232668F8
:100C18005B05B2681A4200D1AAE0B3680025DB0080
:100C280007D410230125A26D1343A365E36D2B435D
:100C3800E3653000FFF7D4FF1022A36D1340034390
:100C480000D0D0E0A36D6A4A1A4002231343A3657B
:100C580023689A68D20766D4227EA07E9203667EB5
:100C6800276B94464203A168F6030192002F01D036
:100C780080277F01E26811436246114331434203F2
:100C880011432269002A00DB87E05200560822003F
:100C98002C32127852000A43611CC97F3A4332430E
:100CA800012905D1002800D07AE0802149020A43B1
:100CB800616A002905D0E02040000140A06A014394
:100CC8000A43D9684B48E76C01400A43DA602200BE
:100CD80061683C3212788E0FB60794463743012A72
:100CE80009D1606C226C0243A06C3A43024360460F
:100CF8003243104307001A693F48024080203A43B4
:100D08001A614A005208C00582420CD0802212069D
:100D1800914208D039483A4E02683240F026B6036C
:100D2800314011430160072070265A69616B824384
:100D38000A435A615869A26BB043120102435A61CF
:100D48002269002A34D1986A103A02439A6207222B
:100D58005B69134099423AD10023E365A36D043AD5
:100D680093431A0001231343A365280005B0F0BD7F
:100D7800B26824490A401343B360234B23491868D7
:100D8800FFF7CCF9013040000390039B002B00D102
:100D980043E7039B013B0393F7E78026B60376E717
:100DA8002020A66D3043A065E06D0143E1657FE733
:100DB800802080038242CAD11C209A6AE269013AE3
:100DC800920002402C3890400200206EBDE71222AB
:100DD800A36D012593431A0010231343A365E36D04
:100DE8002B43E365C1E7A36D01251A43A265BCE760
:100DF800FDFEFFFF0102FEFF02FCFF1F0827014066
:100E0800FFFFC3FFE8FFFF6F00000020400D030055
:100E18007047704710B5806AFFF7FBFF10BD704739
:100E28004023806A10B5826D134383650423C26D25
:100E38001343C365FFF7F3FF10BD0000502310B53F
:100E4800846AA26D1A422CD1A26DB133FF331343C9
:100E5800A365C02320681B01C2681A4214D1A37E6F
:100E6800002B11D103681B070ED5FFF7B9FE002828
:100E78000ED10C21226853688B435360A36D0E4A30
:100E88001A4001231343A3652000FFF7C1FF10BDDB
:100E98002023A26D1343A3650123E26D1343E36589
:100EA800F2E7A36DDB0603D52000FFF7B8FFEEE7F6
:100EB800236D5B6B9847EAE7FEFEFFFF0023F0B562
:100EC80087B00593030054331A7805000E000220FA
:100ED800012A00D1C3E001241C702868FFF780FEB6
:100EE800002800D0F9E004222F6973689743802214
:100EF800019312069446019A3368022A00D1C2E08F
:100F08005903490B2A68029167450FD1906A01433A
:100F18009162B16854691802734E014031408443AC
:100F280021435161002B64DB002095E01F21019FC4
:100F38000F40BC460F2761468F40F9430391296E45
:100F4800B9430F000299002914D1980E1F310840A7
:100F580061468840019907438908E86901312F668D
:100F68008142D6D864469900090FA140906A039C33
:100F78002040CCE72342EBD1022120000B42E7D1ED
:100F8800080049180B42E3D101301907E0D40130B9
:100F9800D906DDD401309906DAD401305906D7D400
:100FA80001301906D4D40130D905D1D401309905BE
:100FB800CED401305905CBD401301905C8D401303D
:100FC800D904C5D401309904C2D401305904BFD41E
:100FD80001301904BCD40130D903B9D401309903C4
:100FE800B6D480211800C90208400B42B0D01220A4
:100FF800AEE7E0243D4A3E48116864040C40834251
:101008001AD180231B0419428ED111683948014036
:1010180021431943384B116018683849FFF77EF8A7
:10102800431C0C2058430590059B002B00D17BE7FF
:10103800059B013B0593F7E73148834211D1802690
:10104800080076043040314200D06DE71168294B22
:10105800194021430E431660002354352B7007B006
:10106800F0BD2848834200D05EE780230800DB03F8
:101078001840194200D057E711681E4E31402143ED
:101088000B431360E8E7674505D128685903826A6E
:10109800490B8A438262002B00DB45E7134A144858
:1010A8001168834208D1A02310685B041940114BD2
:1010B80003401943116037E71148834203D1C02325
:1010C80010681B04F2E70F48834200D02CE7C020C9
:1010D8004004014013680748EAE72023AA6D20006E
:1010E8001343AB65B8E7C04600FFFF070827014078
:1010F800001000B0FFFF3FFE00000020400D03007D
:10110800004000B8002000B470B504000068FFF784
:1011180067FD002801D1002070BD23689A689207F6
:1011280005D49A680F49114010220A439A60FFF7C4
:1011380051FD0426050023689B683342EBD0FFF776
:1011480049FD401B0228F6D923689B683342F2D038
:1011580010230120A26D1343A365E36D0343E365E8
:10116800DAE7C046E8FFFF7F0023F7B504000193E4
:10117800036801209A68024201D00020FEBD9968E8
:10118800224A114207D01023A26D1343A365E36DD1
:101198000343E365F2E79A681D4D2A4010439860BF
:1011A8001C4B1B681B0223D4637E012BE5D0FFF781
:1011B80011FD01260700226813683342DDD19368C8
:1011C800334203D193682B4033439360FFF702FD0A
:1011D800C01B0228EFD923681B683342EBD11023C8
:1011E800A26D01201343A365E36D1E43E665C5E7C1
:1011F800094B0A491868FEF791FF01300190019BDD
:10120800002BD1D0019B013B0193F8E71700008028
:10121800E8FFFF7F0827014000000020400D030081
:10122800F8B5040000680D001600FFF7D9FC02238A
:10123800002840D1270054373A78012A3BD00122B0
:101248003A702368D96811420CD19968114205D0C7
:101258009A681A49114002220A439A600122D96801
:101268000A43DA602000FFF77FFF031E23D1A26D37
:1012780013491140802252000A43A265E065114AD1
:10128800206D2168C262104A0263104A42631C2220
:101298000A603B704A68103313434B602A003300DE
:1012A800403100F075F90300206804498268114054
:1012B80004220A4382601800F8BDC046E8FFFF7F99
:1012C800FEF0FFFF450E00081D0E0008290E00085D
:1012D800036870B50400012099689A68024201D138
:1012E800002070BD02221142FAD105219D680D40EF
:1012F800012D1FD19968134801400A439A600322BF
:101308001A60FFF767FC060023689B682B42E7D04A
:10131800FFF760FC801B0228F6D923689B682B42E4
:10132800F2D01023A26D01201343A365E36D1D4382
:10133800E565D6E71023A26D1343A365E36D034368
:10134800E365CEE7E8FFFF7F70B5060054363378D3
:1013580005000224012B25D001233370FFF7D4FEAA
:10136800041E1DD1286D831DDB7F022B07D100F0E1
:1013780059F9041E03D04023AA6D1343AB6510210D
:101388002A68280053688B435360002C0CD1FFF760
:101398009FFF041E0BD001212A68D3688B43D360BA
:1013A80000233370200070BDFFF792FFF3E7AB6DA9
:1013B800024A1A4001231343AB65ECE7FEFEFFFF28
:1013C80030B5FF2503242A000440E400A240890127
:1013D8002940D243A140C3B200280ADBC0240B4BEA
:1013E80080088000C018A40003591A401143015115
:1013F80030BD0F200340083B05489B089B001B1885
:10140800D86902401143D961F2E7C04600E100E023
:1014180000ED00E0002805DB1F2318401E3B834039
:10142800014A13607047C04600E100E08022431E75
:101438005204012093420DD2C021074A0748536045
:10144800036A09061B021B0A0B43036200200723D9
:10145800906013607047C04610E000E000ED00E0C7
:10146800F0B5846CC56C6560046D002C02D0446DC9
:10147800856D65601C25046C084E25400124AC4030
:1014880077683C437460046863608368102B02D1FA
:10149800A260E160F0BDA160E260FBE700000240ED
:1014A80010B50400036C094A9B089B189B00436411
:1014B80003681421D8B20838FEF730FE044BA36441
:1014C8001F2318401E3B8340E36410BD00820010B8
:1014D8008008024070B504000120002C49D025681E
:1014E800274B1421E818FEF719FE02238000A61DD9
:1014F8002064F3772B68234AE16813402B60A368C4
:101508002A680B43216920000B4361690B43A169D9
:101518000B43E1690B43216A0B4313432B60FFF72D
:10152800BFFF8023A268DB019A4201D100236360D8
:101538003F236268616C13400B60E06CA16C013A58
:101548004860032A16D8104A104899180322013B0C
:101558001340023A9A40A2651300002289002165CF
:1015680060650A60436000200123E0630534F37777
:10157800E07770BD002323656365A365F3E7C04684
:10158800F8FFFDBF0F80FFFF3F82001040090240B7
:10159800F7B5451D0193EE7F04000220012E34D0DB
:1015A8000138E877A71DFE7FB4466346F6B2009679
:1015B8000026834231D10130F8772568E663286830
:1015C800009B98432860019B2000FFF749FF226B8E
:1015D8002368B2421AD00E2219680A431A60626C54
:1015E8001168C90304D580211068490001431160BE
:1015F800226D002A04D0802110684900014311603F
:101608000122002019680A431A60FEBD04211A68E5
:101618008A431A6019680A22DFE78023E363EE77BA
:10162800F3E700000300F0B50120002B09D0981D56
:10163800C27F5C1D022A05D00422DA630023012040
:10164800E377F0BD0E2519685E6C0A68AA430A6044
:101658003268114D2A40326001220E689446964342
:101668000E601C211A6C0D4E114062468A40776844
:101678003A437260D96C9A6C51601A6D002A05D091
:101688001168294011605A6D9B6D53600123C3771F
:101698000020E077D5E7C046FFFEFFFF00000240CC
:1016A800F8B5811DCB7F022B04D00423C363033B11
:1016B8001800F8BD0E240268154D1368076CA34383
:1016C8001360012314689C431460446C22682A4008
:1016D80022601C243C40A3400E4A566833435360A2
:1016E800C26C836C5A60036D002B05D01A682A40BF
:1016F8001A60436D826D5A6001230024CB77431D25
:10170800DC77826B1300A242D2D090472300CFE748
:10171800FFFEFFFF00000240F8B51C210427046CFF
:10172800264A21403C008C40166803681D68264202
:101738000FD03D420DD01968890602D41968B94303
:10174800196053681C43036B5460002B1BD09847E7
:1017580019E002273C008C40264215D03D4213D0A8
:101768001968890606D40A251968A9431960012150
:10177800831DD97753681C4354600022431DDA77D0
:10178800C36A9342E3D1F8BD082427008F403E4244
:10179800F9D02542F7D00E251C68AC431C60012304
:1017A8001D008D402900546821435160821DC36388
:1017B800D3770022431DDA77436BE2E7000002404B
:1017C8000630C07FC0B27047C06B70470020054B21
:1017D8005A69824205DA044A9A60044A9A6058694A
:1017E800C00F70470020024023016745AB89EFCD49
:1017F8008022044B120659690A435A615869C0434A
:10180800C00F704700200240F8B504008027FFF79A
:10181800E1F97F020619124D2B693B420BD12A6967
:10182800104B11001048194028611A4209D00F4B7B
:101838000120596004E0FFF7CDF9B042EBD3032053
:10184800F8BDFFF7C7F980262418F6022B6918009F
:1018580030403342F4D0FFF7BDF98442F6D8EEE7C2
:1018680000200240FA830000FB830000D802002019
:10187800F7B5174E0193337804000D00022000924B
:10188800012B1ED00123FA203370002380007360DF
:10189800FFF7BAFF002812D10E4F012C12D17B6935
:1018A80023437B61009B2B60BFF36F8F019B6B60B1
:1018B800FA208000FFF7A8FF7B69A3437B61002320
:1018C8003370FEBD2800009902F08AFCF0E7C0469C
:1018D800D802002000200240044A05485369C90084
:1018E80003401943034B19435161704700200240DC
:1018F80007E0FFFF02000100F7B5214F05003B7824
:1019080002240191012B1AD00123FA203B700023F5
:1019180080007B60FFF778FF041E0ED104236B6004
:101928002B68042B0DD1FA20164A174B51698000F9
:101938000B435361FFF768FF040000233B7020004E
:10194800FEBD0123019A5B421360AE68AB68EA688A
:101958009B18B3420CD968683100FFF7BDFFFA2025
:101968008000FFF751FF002808D00400019B1E608B
:101978000221044A53698B435361DEE70136E5E7E8
:10198800D802002000200240040001000023F0B526
:1019980085B00A681400DC4001D105B0F0BD01250E
:1019A80014009D402C4001942A4200D18EE04A68E0
:1019B8005E0094460322644622400324B440E44374
:1019C8000294541E012C2AD88768029C2740CC68B0
:1019D800B4403C43846044680127AC432500644616
:1019E80024093C409C402C434460C568029C254027
:1019F8008C68B4402C43C460022A12D1DC08072545
:101A0800A4000419276A03940F241D40AD00AC40BC
:101A1800A7430C69AC402743039C276201E0032AD3
:101A2800E3D10468029DB24025402C0014430460B1
:101A3800C0246246A402224248D0254A03259C08B5
:101A4800A400A4180F221D40ED00AA40A027266E6E
:101A5800FF0596430022B8420CD01E4F0132B8420F
:101A680008D01D4F0132B84204D01C4F0132B84291
:101A780000D00232AA40674632432266144C019ACB
:101A88002668019DD2433543FF0201D43500154035
:101A9800674625606668019D3543BF0201D435005D
:101AA8001540674665600E4C019DE66F3543BF03E0
:101AB80001D4350015406746E5670A4C019EE56F7D
:101AC8002E43FF0301D415402E00E667013360E77B
:101AD800001802400004005000080050000C00509C
:101AE800081802400418024000690840431E984143
:101AF800C0B27047002A01D0816170478162FCE75B
:101B0800426913000B401B049143194381617047DC
:101B18007047000070B5084D0400EB68184202D009
:101B2800E86002F08DF82B69234203D020002C6175
:101B3800FFF7EEFF70BDC0460018024070B5040004
:101B48000120002C17D02368124A07251A60124A70
:101B58001A6062685A60A2689A60FFF73BF806004C
:101B68002368DA68100028402A4205D11969E2681A
:101B780091420CD01A6170BDFFF72CF8801B3128F8
:101B8800EED92368DB682B42EAD00320F3E7034A47
:101B98001A60F0E7CCCC000055550000AAAA000056
:101BA8000368024A00201A607047C046AAAA0000CB
:101BB80010B5114C1149236802000B400343236000
:101BC800802300209B009A420ED10D4B0D491868C6
:101BD80006235843FEF7A2FA8022431CD20061690B
:101BE80008001040114200D110BD002B01D0013B6C
:101BF800F5E70320F8E7C04600700040FFF9FFFF53
:101C08000000002040420F00F0B5040085B0002815
:101C180023D00368DB0710D423689B075ED42368AE
:101C28001B0700D5C3E023685B0700D5F4E0E36930
:101C3800002B00D07AE1002029E03822AF4DAB68B4
:101C48001340EA68102B0AD1D243930709D12B68B5
:101C58009B03E1D56368002BDED1012017E0082B38
:101C6800F5D0802263685202934212D12A68134346
:101C78002B60FEF7AFFF80270600BF022B683B42B0
:101C8800CAD1FEF7A7FF801B6428F7D9032005B047
:101C9800F0BDA021C9028B4208D180232968DB024C
:101CA8000B432B602B681A432A60E2E72A689449A1
:101CB8000A402A602A6893490A402A60002BD8D132
:101CC800FEF788FF80270600BF022B683B42A3D09F
:101CD800FEF780FF801B6428F7D9D7E73823874DA4
:101CE800AA681340EA68102B28D103210A40022A67
:101CF80026D12A68520502D5E268002AADD0696863
:101D080062698148120201400A436A60002B0DD1C2
:101D18002B687E4A1340226913432B602B687C4A48
:101D28009B045B0FDA4013007A4A13607A4B1868F9
:101D3800FEF708FF002800D171E78EE7002BD8D006
:101D4800E368002B20D02B68704A80271340226953
:101D5800FF0013432B6080232A685B0013432B602A
:101D6800FEF738FF06002B683B4207D06A686369B4
:101D780065491B020A4013436B6050E7FEF72AFFD0
:101D8800801B0228EFD981E72B68644A802713401B
:101D98002B60FEF71FFF0600FF002B683B4200D1B7
:101DA8003DE7FEF717FF801B0228F6D96EE73822B9
:101DB800524DAB681340182B08D12B6E9B0700D4EB
:101DC80031E7A369002B00D02DE746E7A26901237C
:101DD800002A10D02A6E022713432B66FEF7FAFE5C
:101DE80006002B6E3B4200D01DE7FEF7F3FE801B7A
:101DF8000228F6D94AE72A6E02279A432A66FEF78E
:101E0800E9FE06002B6E3B4200D10CE7FEF7E2FE2E
:101E1800801B0228F6D939E73822384DAB681340C1
:101E2800202B08D1EB6D9B0700D400E7A368002B9B
:101E380000D0FCE611E780220021EB6B52050091EF
:101E4800134208D1EB6B1343EB63EB6B1340039323
:101E5800039B012300938027314E7F0033683B4268
:101E680015D0A368012B22D1EA6D1343EB65FEF769
:101E7800B1FE02270600EB6D3B4238D0009B012BD8
:101E880000D0D4E6EB6B274A1340EB63CFE6336808
:101E98003B433360FEF79EFE019033683B42E0D13E
:101EA800FEF798FE019BC01A0228F6D9EEE6EA6D05
:101EB800052B05D1013B1343EB65EA6D0123D4E7FC
:101EC80001218A43EA65EA6D03318A43EA65002BFA
:101ED800CDD1FEF77FFE02270600EB6D3B42CDD049
:101EE800FEF778FE104B801B9842F6D9CEE6FEF737
:101EF80071FE0D4B801B9842BDD9C7E60010024009
:101F0800FFFFFEFFFFFFFBFFFF80FFFFFFC7FFFF95
:101F18000024F4000000002008000020FFFEFFFF5E
:101F280000700040FFFFFFEF8813000038213F4D8D
:101F3800AA680A40102A53D03D4A022B38D12B6890
:101F4800802713402B60FEF745FE0600BF042B6870
:101F58003B4227D1616A236AEA680B4335498026E8
:101F68000A401343E26AB6041343226B1343A26A7E
:101F780012021343EB6080232A685B0413432B602F
:101F88008023EA685B051343EB60FEF723FE040039
:101F98002B68334200D04EE6FEF71CFE001B0228D9
:101FA800F6D973E6FEF716FE801B0228CFD96DE638
:101FB8002B68802613402B60FEF70CFE0400B60445
:101FC8002B6818003040334204D1EB681A4A13409A
:101FD800EB605CE6FEF7FEFD001B0228F0D955E633
:101FE800012B00D139E60322EB68216A1A408A42A4
:101FF80000D032E67022616A1A408A4200D02CE68C
:10200800FE21A26AC90119401202914200D024E6B9
:10201800F822E16A92031A408A4200D01DE6226B38
:102028005B0F5B07934200D105E616E600100240FD
:10203800FFFFFFFE8C80C11FFCFFFEEF382370B549
:102048001E4CA2681A4205D123681D489B045B0FE9
:10205800D84070BDA2681A40082A2AD0A2681A403F
:10206800102A1AD1E368E168DB434906490F7F2546
:1020780001319B070CD1E36812481B0A1D40FEF78B
:102088004DF8E1686843490F0131FEF747F8E0E78A
:10209800E3680B481B0A1D40F1E7A2681A40202A92
:1020A80009D0A26800201340182BD2D1FA20C00111
:1020B800CFE70448CDE780200002CAE700100240BD
:1020C8000024F40000127A00F7B504000D0000287F
:1020D80001D10120FEBD07274A4E33683B408B42A1
:1020E8002AD321688B073BD4CB0748D4072733680A
:1020F8003B40AB420AD93368BB432B433360FEF7FE
:1021080069FD019033683B40AB426BD123683E4D7B
:102118005B076FD4FFF792FFAB683C4A1B051B0FA8
:102128009B009B581F221340D840394B1860394BED
:102138001868FEF707FDCDE73368BB430B433360F0
:10214800FEF748FD019033683B40AB42C9D0FEF72B
:1021580041FD019BC01A304B9842F4D90320B9E7DE
:10216800294A4B0704D5E0239068DB0103439360B9
:1021780093682A480340A06803439360B4E7626801
:10218800214F012A19D13B689B03A2D50721BB68BF
:102198008B431343BB60FEF71DFD01903823BA68DB
:1021A8001A406368DB009A42A0D0FEF713FD019B3A
:1021B800C01A194B9842F1D9D0E7022A03D13B68DB
:1021C8009B01E3D485E7002A03D13B685B05DDD496
:1021D8007FE70223032A03D1396E1942D6D178E763
:1021E800F96DFAE7FEF7F6FC019BC01A0A4B984214
:1021F80088D9B3E7AB680A4A1340E2681343AB6077
:1022080088E7C0460020024000100240F84100085C
:10221800000000200800002088130000FFF0FFFFE6
:10222800FF8FFFFF064B074A9B685B045B0F9B0011
:102238009B581F221340044A1068D8407047C04674
:10224800001002403842000800000020F0B50500E8
:102258002B68002085B09B033BD58022484C520553
:10226800E36B0090134208D1E36B1343E363E36B22
:1022780013400393039B012300938027414E7F0063
:1022880033683B433360FEF7A5FC019033683B425B
:1022980011D0E26DC02311009B003B4E19401A4239
:1022A80002D06B6999424DD1E36D00201E406B69E5
:1022B8001E43E66506E0FEF78DFC019BC01A022866
:1022C800E4D90320009B012B03D1E36B2F4A134071
:1022D800E3632A68D30706D5032429494B6DA34332
:1022E8006C6823434B65930606D52549284C4B6DEE
:1022F8002340AC6823434B6553040FD520492C6910
:102308004B6D9B009B0823434B658023DB059C4258
:1023180004D18023CC685B022343CB6013050FD51F
:10232800174A1C4C536DE96823400B4353658023BF
:10233800DB01994204D18023D1685B020B43D3604F
:1023480005B0F0BD8023E26DE06D11005B02034330
:10235800E365E36D104831400340E365E165D30769
:10236800A2D5FEF737FC07000222E36D13429BD18A
:10237800FEF730FC094BC01B9842F5D9A1E7C046CF
:102388000010024000700040FFFCFFFFFFFFFFEF5E
:10239800FFCFFFFFFF3FFFFFFFFFFEFF8813000097
:1023A8000122036A70B593430362036A164A4468BC
:1023B800856915400A681543022293438A681343C6
:1023C800124A904205D0124EB04202D0114EB0428D
:1023D80013D10826B343CE6833430426B34390424F
:1023E80005D00B4A904202D00A4A904205D10A4AC7
:1023F8008E6922404C69344314434A6844608561BD
:102408004263036270BDC0468CFFFEFF002C014092
:102418000044014000480140FFFCFFFF036A174ADF
:1024280070B513400362036A154D4268C4692C40B5
:102438000D682C43134D2B408D682D022B43124DF4
:10244800A8420ED1114D1D40CB681B022B43104DE5
:102458002B40104D4E6915408A69324312012A43B8
:1024680005E00D4DA842F4D00C4DA842F1D04260D1
:102478004A68C461C263036270BDC046FFFEFFFFC5
:102488008CFFFEFFFFFDFFFF002C0140FFF7FFFF61
:10249800FFFBFFFFFFCFFFFF004401400048014062
:1024A800036A124A30B513400362026A104C43684B
:1024B800C56925400C68240225430E4C22408C68CF
:1024C800240322430C4CA04205D00C4CA04202D05D
:1024D8000B4CA04204D10B4C23404C69A40123436C
:1024E80043604B68C5610364026230BDFFEFFFFFC4
:1024F800FF8CFFFEFFDFFFFF002C0140004401407E
:1025080000480140FFBFFFFF036A70B5104E114C31
:1025180033400362026A4368456D25400C682543D1
:102528000D4C22408C68240422430C4CA04205D058
:102538000B4CA04202D00B4CA04203D14C69334053
:102548002402234343604B6845658365026270BD7E
:10255800FFFFFEFF8FFFFEFFFFFFFDFF002C014086
:102568000044014000480140036A124A30B5134054
:102578000362026A104C4368456D25400C682402CA
:1025880025430E4C22408C68240522430C4CA04263
:1025980005D00C4CA04202D00B4CA04204D10B4CED
:1025A80023404C69A402234343604B684565C365D7
:1025B800026230BDFFFFEFFFFF8FFFFEFFFFDFFF6F
:1025C800002C01400044014000480140FFFFFBFF90
:1025D8000200030001203D321178814218D1022106
:1025E80011701B68DA680243DA600C4A934202D021
:1025F8000B4A93420DD19A680A4900200A40062ADC
:1026080006D007398A4203D0012219680A431A60A2
:1026180070471A68104318600020F9E7002C014041
:10262800000400400700010070470000194A10B577
:102638000368904202D0184CA04208D17024A343EA
:102648004C68234390420BD0134CA04208D0134C43
:10265800A04205D0124CA04202D0124CA04203D195
:10266800114C2340CC6823438024A3434C69234363
:1026780003608B68C3620B688362904205D0084B85
:10268800984202D0074B984201D10B69036301239A
:10269800436110BD002C01400004004000200040B0
:1026A8000044014000480140FFFCFFFF70B50400F2
:1026B8000120002C23D025003D352B78DAB2002BE1
:1026C80005D123003C3320001A70FEF7E3F80223FB
:1026D8002B702068211DFFF7A9FF2200012300208D
:1026E8004832137047340A3A137053709370D3709A
:1026F800137153719371D371137223702B7070BD62
:1027080070B504000120002C23D025003D352B781E
:10271800DAB2002B05D123003C3320001A70FFF7F2
:1027280083FF02232B702068211DFFF77FFF220003
:10273800012300204832137047340A3A137053704B
:102748009370D370137153719371D3711372237093
:102758002B7070BD1022036A70B593430362026A3E
:10276800154C4368856925400C68240225432024BC
:10277800A2438C6824012243104CA0420FD180242C
:10278800A2431400CA68120122434024A2430C4EFB
:102798004C691E408B6923439B00334305E0094C79
:1027A800A042F4D0084CA042F1D043604B68856148
:1027B8008363026270BDC046FF8CFFFE002C01409F
:1027C800FFF3FFFF0044014000480140F8B507004F
:1027D8003C373B7804000D0016000220012B0CD07A
:1027E800013838700C2A51D008D8042A2DD0082A6C
:1027F8003CD0002A17D000233B70F8BD102A56D0D1
:10280800142AF8D12068FFF7AFFE8022236812014E
:10281800596D0A435A655A6D2D490A405A652A6905
:10282800596D120251E02068FFF7BAFD08222368AB
:1028380099690A4304219A619A698A439A619A6953
:1028480029690A439A610020D5E72068FFF782FFCB
:1028580080222368120199690A439A619A691C497E
:102868000A409A612A6999691202EAE72068FFF723
:10287800D5FD04212368DA691643DE61DA698A43E3
:10288800DA61DA6929690A43DA61DCE72068FFF767
:1028980007FE802223681201D9690A43DA61DA69DE
:1028A8000B490A40DA612A69D9691202EBE7206804
:1028B800FFF72AFE08222368596D0A4304215A6546
:1028C8005A6D8A435A655A6D29690A435A65BAE7A7
:1028D800FFFBFFFF1F2310B5012419408C408A40DD
:1028E800036AA3430362036A1A43026210BD00002D
:1028F80010B50400002906D1020001203E321378E9
:10290800834249D010BD0300042929D101203F3357
:102918001A788242F6D102221A702268D3680B43D1
:10292800D36020680122FFF7D5FF23682D498B4229
:1029380049D02D4A934246D02C4A934243D02C4A40
:10294800934248D19A682B4900200A40062AD9D0D8
:1029580007398A42D6D0012219680A431A60D1E79A
:1029680008290FD140331B780120013B5A1E93419F
:10297800DBB2002BC6D10223082913D12200403232
:102988001370CAE70C2901D14133ECE7102901D1B2
:102998004233E8E74333E6E7022313702268D0683E
:1029A8000343BDE70C2906D1220041321370226887
:1029B8001023D068F4E7102903D142340120237092
:1029C800A0E74334FAE78022586C120202435A64A3
:1029D8008B42B4D1B6E70122196800200A431A6075
:1029E80090E7C046002C01400044014000480140E7
:1029F800000400400700010010B5FFF779FF10BD83
:102A080030B5EFF31084012282F31088C0250168E5
:102A18000B68AB430B6084F31088EFF3108182F3EB
:102A280010880268044C93682340936081F31088EF
:102A380020238830036030BDFFFF7FFF30B5EFF300
:102A48001084012282F310880168134D0B682B4013
:102A58000B6084F31088EFF3108182F3108802680A
:102A68000E4C93682340936081F31088C36E012B4A
:102A78000AD1EFF3108183F31088102402681368D9
:102A8800A343136081F31088030020228C331A605B
:102A98000023C366436730BDDFFEFFFFFEFFFFEF85
:102AA800F7B50500883513002A6804000220202A9B
:102AB80032D1013800292FD0002B2DD08022A068D8
:102AC8005201904206D12269002A03D10132100036
:102AD800114221D12200260054322165002713809B
:102AE80053802122E06F903637602A60B84214D0B4
:102AF800226887630192114AC262114A0263114A2D
:102B08004263019A2832FEF743FDB84205D01023EC
:102B180001203360DB182B60FEBD402223681A6257
:102B2800EFF31081012383F3108822687F339068C4
:102B38000343936081F310880020EDE7F92B000828
:102B48004B2C00085B2C00080300020080218C320B
:102B5800883370B51B6815680268040092680A42D9
:102B680020D0212B1ED1EFF31080203B83F3108857
:102B7800226893688B43936080F31088E06F002885
:102B88000DD0FEF74FFD002809D0E06FFEF71CFEC0
:102B9800202804D11023903423601D3870BD2000F4
:102BA800FFF72EFF4021236800209B680B42F5D0D9
:102BB800222DF3D1EFF31080012383F31088250031
:102BC80004CD93688B43936080F31088E86F0028E6
:102BD80008D0FEF727FD002804D0E86FFEF7F4FDC3
:102BE8002028D7D02000FFF729FF0020D6E770471C
:102BF80003001B6870B51A6820231100806A194009
:102C08001A421AD1030056331980EFF310840122B7
:102C180082F31088802501688B68AB438B6084F34E
:102C28001088EFF3108182F310884023026810683F
:102C38000343136081F3108870BDFFF7D8FFFBE7EB
:102C4800704710B5806AFFF7FBFF10BD70477047EB
:102C5800704770B5846A2300220088338C321B6861
:102C6800156822689268120608D5212B06D1230020
:102C78000022563320001A80FFF7C2FE23689B68A3
:102C88005B0608D5222D06D1230000225E332000E2
:102C98001A80FFF7D3FE220010239032116820001B
:102CA8000B431360FFF7D4FF70BD806A0023020056
:102CB80010B55E321380083A1380FFF7C9FF10BDC4
:102CC80070470000F7B50168C04DCB6904000A6879
:102CD80088682B4210D120252B4200D19AE080260B
:102CE800760515400640354300D193E0636F200018
:102CF800002B00D083E083E0B54D0540AC46664626
:102D0800B44D1540354300D184E001252B4207D04E
:102D1800D60505D526000D62903637683D433560E7
:102D28002500022690350195334207D0C50705D501
:102D3800019D0E622F68B6193E432E600426334269
:102D480009D0C50707D527000E6290373E683500C1
:102D580002262E433E60082633420AD020276546C5
:102D680017402F4305D027000E6290373D682E4349
:102D78003E60802726003F0190363B4206D0550131
:102D880004D50F6220213768394331603168002942
:102D980036D020210B420AD0114080225205104023
:102DA800014304D0636F002B01D0200098472268AC
:102DB800019B40271B68966828223E40134020004C
:102DC8001E4322D0FFF73AFE23689B683B4218D087
:102DD800EFF31081012383F31088250004CD936855
:102DE800BB43936081F31088E86F002809D07A4BC1
:102DF8008363FEF755FC002802D0E86F836B984781
:102E0800F7BD2000FFF724FFFAE7FFF721FF019B3A
:102E18001E60F5E7E56E012D00D09EE010263342D6
:102E280000D19AE0324200D197E00E628B684022CE
:102E380018001040134256D0201DC36F19684B6804
:102E48009BB2002BDCD027005C373F889F42D7D944
:102E580027005E373B80096820230F001F40019739
:102E6800194232D1EFF3108785F3108821685B4E41
:102E7800096831402668316087F31088EFF3108CB9
:102E880085F310882768B968A943B9608CF310885E
:102E9800EFF3108C85F310882768B9689143B960FF
:102EA8008CF3108822008C321360019BE366EFF3E9
:102EB800108185F3108822680F351368AB431360BF
:102EC80081F31088C06FFEF7ADFB02232200236751
:102ED80023005C325E331B881188C91A89B220002E
:102EE800FFF7EEFE8CE722005E32138812889BB251
:102EF800002A00D184E722005C321188C91A89B2FD
:102F0800002900D17CE7EFF3108785F31088226849
:102F1800334E13683340136087F31088EFF310873C
:102F280085F3108822682F4E93683340936087F3A7
:102F38001088230020228C331A60E0666067EFF364
:102F4800108085F31088102522681368AB4313603E
:102F580080F3108802232367C1E780256D032B4285
:102F680006D0460204D520000D6200F03FFB47E77B
:102F780080210B4207D080252D04114028400843AA
:102F880001D0A36FB3E640210B4216D00A4214D0F9
:102F9800EFF31080012383F31088226813688B43B2
:102FA800136080F310882300202288331A600023DE
:102FB8002000A367FFF71BFE22E7190214D5510072
:102FC80012D5200000F014FB1AE7C0460F080000D5
:102FD8000100001020010004B32C0008FFFEFFFFD1
:102FE800DFFEFFFFFEFFFFEFDB0100D408E7002A4A
:102FF80000DB05E7200000F0FAFA01E70123806A08
:1030080010B50367C36E012B06D103005C33198822
:103018004908FFF755FE10BDFFF719FEFBE7000052
:1030280003001B6820221B6870B51900806A1140D4
:10303800134234D103005E331980EFF31085012366
:1030480083F3108804681D4E21683140216085F3A0
:103058001088EFF3108583F310880468A1689943FA
:10306800A16085F31088EFF3108483F3108840255E
:1030780001688B68AB438B6084F3108803008C3342
:103088001A60C36E012B0AD1EFF3108183F3108805
:10309800102402681368A343136081F31088002387
:1030A8000367C36E012B05D103005C331988FFF752
:1030B80007FE70BDFFF7CAFDFBE7C046FFFEFFFF36
:1030C80070B504002569A168026829436569C36968
:1030D80029431068484D194328400143116051683D
:1030E8004648256A0140E06801435160A16990683B
:1030F8002943434D284001430F209160D16A814301
:10310800606A0143D1623F498A4215D103213E4A90
:10311800526D0A408021013A0902022A5FD83B48D1
:10312800805C8B4214D0082857D8FCF7EDFF0C566A
:103138005456515656563B0035498A424DD1802245
:10314800120293424DD0FFF76DF800284DD02BE0C6
:10315800082842D8FCF7D8FF4541084105414141BC
:103168000900FEF76BFF3EE02A4B626A2A495200CB
:10317800515A1800FCF7D2FF656840006B08C01868
:103188002900FCF7CBFF0200244B103A9A4224D8BE
:103198000F23020000079A4393B2400F2268184396
:1031A800D06022E080200002636A1B4A5B00995AC3
:1031B800FCF7B4FF65686B08C0182900FCF7AEFF80
:1031C8000200164B103A9A4207D82368D8600CE0E0
:1031D800FEF734FFB9E70F48E6E7012006E08B4227
:1031E800B1D1FFF71FF8031EBFD100200C4BA36617
:1031F80000236367A36770BDF369FFCFFFCFFFFFAD
:10320800FFF4FF1100380140001002405842000846
:10321800004400400024F4005C420008EFFF000076
:1032280001000100836A30B5DA0706D50168284C29
:103238004A682240C46A22434A609A0706D5016850
:10324800244C4A682240046B22434A605A0706D538
:103258000168214C4A682240446B22434A601A079D
:1032680006D501681D4C4A682240846B22434A6097
:10327800DA0606D501681A4C8A682240C46B2243D4
:103288008A609A0606D50168164C8A682240046C42
:1032980022438A605A0610D50168134D4A68446C67
:1032A8002A4022434A6080225203944205D14A6848
:1032B8000E4C2240846C22434A601B0606D50268E5
:1032C8000B4953680B40C16C0B43536030BDC0467B
:1032D800FFFFFDFFFFFFFEFFFFFFFBFFFF7FFFFF7D
:1032E800FFEFFFFFFFDFFFFFFFFFEFFFFFFF9FFF86
:1032F800FFFFF7FFF7B5802704000D0016000193C4
:103308003F012268D3692B405B1B59424B41B342B2
:1033180001D000202AE0089B0133F3D0FDF75AFCC6
:10332800019BC01A089B984201D8002B1FD1EFF3CC
:103338001080012282F310882168204D0B682B40F1
:103348000B6080F31088EFF3108082F310882168F7
:103358008B6893438B6080F3108822002023883287
:10336800136053600023032084342370FEBD0421BE
:1033780023681A680A42C4D0DA693A42C1D01F6287
:10338800EFF31080012282F3108821680B4D0B683F
:103398002B400B6080F31088EFF3108082F31088C5
:1033A80021688B6893438B6080F310882200202368
:1033B8008832136053609360D4E7C0465FFEFFFF16
:1033C800030073B50026040090331E60FDF702FC6D
:1033D800236805001B681B0719D423681B685B0753
:1033E8000AD58021104B0022009320002B00C9032E
:1033F800FFF780FF002815D1220000202023883203
:1034080013605360E0662067843420700BE08021ED
:10341800054B32000093890303002000FFF76AFF81
:103428000028DAD0032076BDFFFFFF0170B5041E27
:1034380001D1012070BD050088352B68002B04D10F
:10344800020084321370FDF7D1FA24230121226887
:103458002B60136820008B431360FFF731FE0128AF
:10346800E7D0A36A002B02D02000FFF7DBFE236819
:1034780007495A6820000A402A215A609A688A43F4
:103488009A60012219680A431A60FFF799FFD1E789
:10349800FFB7FFFFF8B513000200060005005C3215
:1034A80081650F0013802221002290368C3532600E
:1034B8002960011D0400C86F904213D01D49826322
:1034C800C1621D493A0001631C49416321682431E6
:1034D800FEF75EF8002805D0102301203360DB18C2
:1034E8002B60F8BD2369002B0BD0EFF3108101236B
:1034F80083F310882268FF3310680343136081F355
:103508001088EFF31080012383F3108821688A68FC
:103518001A438A6080F31088EFF3108183F31088D0
:1035280022683F3390680343936081F3108800203A
:10353800D7E7C04629300008053000085B2C000892
:1035480003008C3370B51C680223202C25D1013B65
:10355800002922D0002A20D0802384685B019C4265
:1035680005D10369002B02D10133194215D100237B
:10357800C36603685B681B020CD5EFF31085012353
:1035880083F3108880230468DB04266833432360B0
:1035980085F31088FFF77EFF0300180070BD000058
:1035A800F8B5436E0400002B02D10D4B8366F8BDBD
:1035B80003680C4E9F689B680B4D5B0FF05CE95CE1
:1035C800C000FCF735FE23006A3318803B015B0F0F
:1035D800F05CE95CC000FCF72BFE68342080E6E76D
:1035E800010001007C4200087442000870477047DF
:1035F8007047000070B5040084342278030002206C
:10360800012A11D01D002422012688352A601A6853
:1036180011681068B04310600448014000205866E3
:10362800202311602B60207070BDC046FFFFFFDFB4
:10363800F8B50400250084352A7808000223012AF9
:1036480018D0012126002970226888362233336079
:10365800176813688B4313609368DB00D90801432C
:1036680091602000FFF79CFF23681F6020233360D0
:1036780000232B701800F8BDF8B5050084352B78A9
:1036880004000A000220012B18D026002423013848
:1036980028708836336023681F6819688143196069
:1036A800996807480140114320009960FFF778FFA7
:1036B800236800201F60202333602870F8BDC046AF
:1036C800FFFFFFF11022044B1B6819680A431A60B8
:1036D80050221A627047C04640020020F8B5254CB7
:1036E8000121228813004800205A984238D8051C26
:1036F800904200D9151CAAB20131FA29F3D1002051
:103708009B1A834200DD18B21B4C23785A1C227086
:10371800032B24D9194B05211F88194B3FB21E884A
:10372800184B36B21D78FCF783FD03B216481749CB
:103738005843FCF77DFD0A217843FCF779FD6DB20B
:1037480080196843124B134A00B218801178012976
:1037580008D11B88104A1BB2138000232370F8BDC0
:103768000300C9E71278002AF7D11B880B4A1BB25D
:10377800F2E7C046F6020020F9050020EC0500201B
:10378800EA05002017000020E40C0000FF0F0000ED
:10379800EE050020F5050020F2050020F0050020C8
:1037A800F0B50825012602000B4F0C4801390B4BD8
:1037B80089B2994200D1F0BD137858402B0004001B
:1037C8004008344001D0784080B2013BDBB2002B86
:1037D800F5D10132EAE7C04601A0FFFFFFFF000074
:1037E800022310B501241D4A88B011880493128859
:1037F800DB1805930B330693120A02AB5A70184A6A
:103808001970118812889970120ADA70154A07948B
:1038180011881288197112B212125A71124A11883B
:103828001288997112B21212DA71FDF7CFFF01A94D
:1038380004A8FEF761F8002802D0FDF7D9FF0AE0D6
:103848002000029A039B0949FEF712F8041EF4D0DF
:10385800FDF7CEFF0324200008B010BDF4020020BD
:10386800FC050020EC050020EA050020007800088F
:10387800022330B5012487B0154D0293DB1803935A
:103888000A3304932B68059408332B60FDF79EFFD9
:10389800104B2A689A420AD90F4B01A902A82B603B
:1038A800FEF72AF8002802D0FDF7A2FF0CE00B4B28
:1038B80001201A88296812B2D317FDF7D9FF041E10
:1038C800F2D0FDF795FF0324200007B030BDC046B5
:1038D80010000020D877000800700008F6050020C6
:1038E80010B50400A02001222021C005FEF702F92E
:1038F80009490A48A2B2FFF7D3F80948FDF760FF63
:103908000128FAD1043000F011FCA0200022202167
:10391800C005FEF7EFF810BD6A0500204002002040
:10392800E4010020F0B5444D8BB0EB78A9781B0278
:103938000B436C792A795BBA9BB2062128002402D2
:1039480014430093FFF72CFF030ADBB20193C3B2C1
:1039580002933A4B64BA1A88394BA4B25A80394A4E
:10396800127852B29A80384A1278DA80374A128826
:103978001A81374A12885A81364A12889A81364AF9
:103988001288DA81009AA2180A2A23DCAA790299F5
:103998008A421FD1EA7901998A421BD12F492A7894
:1039A8000A706A7803254A7062008A700022681CCF
:1039B800C0B2AE1C0390F6B294422BD8274FA9B2DE
:1039C8003800FFF7EDFE039B7855000AF8543000E5
:1039D800FFF786FF009BFF2B1AD1012C18D1164B3D
:1039E80002999A798A4213D1DB79019A93420FD1CD
:1039F800002405AD12222800194900F0D3FB174E08
:103A08002800FCF779FB844210D3C0B2FFF768FFA7
:103A18000BB0F0BD009810184000185E0132071274
:103A28004F55039DD2B248553500C0E72B5D33553D
:103A38000134E4B2E4E7C046FE050020EE050020AC
:103A4800800600200C00002016000020FC05002045
:103A5800EC050020EA050020F60500206A05002094
:103A680084420008F7B5574CE378A1781B026579C2
:103A78000B4322795BBA9BB2062120002D02154325
:103A88000193FFF78DFE06004F4F062221003800F4
:103A980000F088FBF3B2019A360AF6B26DBABB7130
:103AA800FE710F2A22D1A2799A4212D1E379B34248
:103AB8000FD1ABB2013BF62B0CD8444B1D80FFF75E
:103AC8008FFE002805D16378002B02D00820FFF76D
:103AD80007FFF7BDFF2306213B717B712000FFF72D
:103AE8005FFEB871000A2378F871EDE7019A042A9D
:103AF80016D1A2799A42ECD1E379B342E9D1FA23FB
:103B0800AAB29B009A42E4D8314B324A1D801B88E6
:103B180012689BB25363FFF763FE0028D9D1D5E73B
:103B2800019A28B2052A24D1A2799A42D1D1E379FF
:103B3800B342CED12849ABB25B18284A9BB2934214
:103B4800C7D8274B19880A2309B25843FCF770FBDA
:103B5800244BAAB200B2053A18800F2A00D81D805B
:103B68001A8812B2042AB4DD1B881BB2142BB0DCED
:103B7800D1E7019A062A10D1A2799A42A9D1E3790C
:103B8800B342A6D1144AABB29446144A63449BB2DA
:103B980093429ED8144B1D80BDE7019A072A00D096
:103BA80097E7A2799A4200D093E7E379B34200D02D
:103BB8008FE70E4B0E4A1D800E4B1A60FFF758FE1A
:103BC800ABE7C046FE0500206A050020F40200208D
:103BD800FC0500203C010020E40C0000C81900008E
:103BE800EE050020EC050020EA050020F60500207F
:103BF800D87700081000002010B50E4B0E491A782F
:103C080009888A420ED10D49097808290AD15B78BA
:103C1800032B04D0062B04D1FFF724FF01E0FFF7A4
:103C280081FE10BD002AFCD1044A1278082AF8D176
:103C38005B78EFE7FE050020F40200207E060020F6
:103C480010B5040080282ED1FA210420890000F044
:103C58002FFA3F4C2378012B06D1FA210220490084
:103C680000F026FA00232370A0204021C005FDF7AC
:103C78003BFF012803D1374A137801331370364AC2
:103C880013780133DBB21370052B09D9314B334953
:103C98001878022805D901200870002111701970C0
:103CA80010BDFF20F8E70828FAD103202C4900F0BE
:103CB800FFF9A0202100C005FDF716FF294B2A496E
:103CC8002A4A012827D118700B8829491BB209886C
:103CD800128809B25B1A934210DD264A1378013321
:103CE800DBB21370022BDBD9002123480170234873
:103CF8000170FA2BD4D903231370D1E71F4A137824
:103D08000133DBB21370022BCAD91B49087000209B
:103D180018490870EDE7002018700B881BB2D817F7
:103D28001B18434016489BB2834202D9962313803E
:103D3800B6E70B881BB2D9175B184B40FA219BB228
:103D480049008B4201D96423F1E72823EFE7C046F5
:103D580016000020FA050020F405002017000020B6
:103D680088130000F5050020F2050020140000204B
:103D7800F0050020FB0500200C000020F8050020BD
:103D8800DC050000F8B5FFF79DFC744B1A88744BEE
:103D98001A801A88002A03D01988724A914201D1E0
:103DA80001221A80704B1A88704B1A801A88002AD0
:103DB80003D019886B4A914202D1FA2292001A80E4
:103DC8006B4C1B8822689BB253636A4B00229A5E35
:103DD800694B1A801A88002A03D01A8812B2013255
:103DE80001D10A221A80654B00229A5E644B1A8020
:103DF8001A88002A03D01A8812B2013201D100228F
:103E08001A800120002184465E4A5F4B5F4F136091
:103E18000025585F1D00388008201E5E3888083548
:103E280000B2B04200DA8DE0002900D013603B8870
:103E38001BB2002B01DC00233B802000FEF7C8FBEF
:103E480000212000FEF7D8FD514C04262000FEF783
:103E58007BFE802220004F49FFF772FB4E4DFA226D
:103E68004E492800FDF7DCF9A02000222021C005DA
:103E7800FDF740FE3221002000F01AF9FA21012056
:103E8800490000F015F90320454900F011F9FA211D
:103E98000420890000F00CF90024002000F032F919
:103EA800002809D02800FDF74FFAFFF717FCFA227F
:103EB80028003A49FDF7B4F9012000F023F9002859
:103EC80006D03848FDF76CFE01213748FDF718FE8B
:103ED800022000F017F9002811D0A0203100C005F9
:103EE800FDF70EFEE1230134A4B25B019C4206D922
:103EF8003B88002401331BB23B80FFF7B9FC032049
:103F080000F000F9002802D00222284B1A70300075
:103F180000F0F8F800280BD0022000F0DFF8A0200D
:103F280001223100C005FDF7E5FD0122204B1A7082
:103F3800204B1B78002BB0D0FFF75EFE00231D4AF4
:103F48001370AAE71C4B9D4203D02B0061463E80AC
:103F58005EE7002900D16AE7184B67E70078000898
:103F6800F4020020FFFF000002780008FC05002092
:103F78003C01002004780008EC05002006780008C1
:103F8800EA0500201000002000700008F605002057
:103F980040020020EA0400206C000020F602002005
:103FA800881300002C010020000400500C000020A1
:103FB800160000207E060020E0770008D877000869
:103FC800002370B50C251C00124928005843013302
:103FD8000A185460946054704454062BF5D1FA21A1
:103FE8000D4B89001868FCF799F8802301385B04A9
:103FF80098420DD2C021094A090650600848036A50
:104008001B021B0A0B43036207239460136070BDF5
:10401800FEE7C0469C0600200000002010E000E0FB
:1040280000ED00E01C4A70B51368002B07D0136838
:10403800013B1360002B02D10122184B1A70002299
:104048000C25012616482C005443031959680029E9
:104058000AD0596801395960002905D15E70215C80
:10406800012901D1996859600132062AEBD10D4B1B
:104078001A6801321A6019680B4A914201D100226C
:104088001A600A4A13780133DBB2092B01D813707E
:1040980070BD0023FBE7C046E8060020E4060020C8
:1040A8009C06002094060020FFFFFF7F9806002052
:1040B800030030B5052800D9FEE7012585F31088EF
:1040C8000C2000225843044C2318596099605A70F8
:1040D800055582F3108830BD9C0600200300052892
:1040E80000D9FEE7012282F310880C2058430023F0
:1040F800034A11184B604B70835483F31088704740
:104108009C06002003000020052B09D80C305843DA
:10411800054B00221B185978C8B2012901D15A70E1
:1041280070471000FCE7C0469C06002000280FD00E
:10413800012800D10130012383F310880022054BA8
:104148001860054B1A7082F310881A78012AFCD17E
:104158007047C046E8060020E406002070B5002637
:104168000C4D0D4C641BA410A64209D1002600F08A
:104178002BF80A4D0A4C641BA410A64205D170BD49
:10418800B300EB5898470136EEE7B300EB58984771
:104198000136F2E798420008984200089842000861
:1041A8009C420008002310B59A4200D110BDCC5C97
:1041B800C4540133F8E703008218934200D17047D2
:1041C80019700133F9E70000F8B5C046F8BC08BC1F
:1041D8009E467047F8B5C046F8BC08BC9E46704776
:1041E80001B40248844601BC604700BF19000020A2
:1041F80000000000000000000000000000000000B7
:1042080000000000000000000000000000000000A6
:10421800010000000200000003000000040000008C
:104228000600000007000000080000000900000068
:104238000000000000000000000000000000000076
:10424800010000000200000003000000040000005C
:1042580004020800010002000400060008000A0029
:104268000C00100020004000800000010804020437
:104278000801010101010103070100004443452D24
:10428800323330322D56352E305F48414C00000015
:04429800E100000839
:04429C00B90000085D
:1042A0000024F400010000000400000001000000F0
:1042B000007000084600010180220C4B30B55C699B
:1042C000D20222435A61EFF3108272B64C1CFF34C3
:1042D000401A0D6845500431A142FAD180214902AB
:1042E00018690842FCD182F3108830BD00200240DA
:0400000508000AF9EC
:00000001FF
